:100000000C9430010C9458010C9458010C94580134
:100010000C9458010C9458010C9458010C945801FC
:100020000C9458010C9458010C9458010C949A3972
:100030000C9442320C9458010C9458010C945801C1
:100040000C942D3A0C9458010C94D13B0C941F3C09
:100050000C9458010C9426330C9458010C945801BC
:100060000C9458010C94580172636172676D73654A
:1000700000D40A710B1F0CD10CAC0D5F0E460F3271
:1000800010281134123C136F149815E7164D18B34D
:1000900019301BBB1C681E5620522275247726B4CB
:1000A000280F2B8E2D72303F334A367239F63C6B57
:1000B000408E447B48DD4C795122567C5BE760558D
:1000C00066A76C28732873287328732873287328ED
:1000D000732873000005000A0050007F00A000DCB8
:1000E00000FF0000001900190064009001E803D02F
:1000F00007A00F00001E003C0055006E009200B4E7
:1001000000C300DC00FF0000008813E02E983A8056
:100110003E803E6842204E7869007D00000100026A
:1001200000030006000C001800300048006000903A
:1001300000C0002001800140020003C05D6D03008B
:100140000000000000000080000000FE030D0052CF
:10015000003600FF037F007F007F007F00FF00FF6D
:1001600003FF033F007F007F007C3C3E5E2B3D3F52
:100170002F5B5D3B2C2A225C00040302010001027C
:1001800004030506073F065B4F666D7D077F6F77AB
:100190007C585E79713D74041E703855545C7367E9
:1001A000506D781C0C6A49725B004049526461745E
:1001B000610000E4CBB5A2908072665B5148403983
:1001C000332E2924201D1A171412100E0D0B0A09A4
:1001D00008070605040302016461746100666D741A
:1001E00020005741564500524946460064617461FB
:1001F00000666D742000574156450052494646003E
:1002000000000000240027002A0000000000250054
:1002100028002B0000000000230026002900040411
:10022000040404040404020202020202030303039E
:10023000030301020408102040800102040810207A
:100240000102040810200000000700020100000362
:10025000040600000000000000006306911B8B3DB7
:1002600011241FBECFEFD8E0DEBFCDBF11E0A0E06C
:10027000B1E0EAE4FDE702C005900D92A83BB107AA
:10028000D9F718E0A8EBB1E001C01D92A633B10781
:10029000E1F712E0C0E6D2E004C02297FE010E941E
:1002A0009F3ECA35D107C9F70E94E13D0C94A33E99
:1002B0000C940000FB01DC014150504030F08D9166
:1002C0000590801919F40020B9F7881B990B08953F
:1002D000FB01DC014150504048F005900D92002098
:1002E000C9F701C01D9241505040E0F70895FB014D
:1002F000DC0104C08D910190801921F441505040DF
:10030000C8F7881B990B0895FB01DC0102C001901E
:100310000D9241505040D8F708958F929F92AF921E
:10032000BF92CF92DF92EF92FF920F931F93CF93E2
:10033000DF9370E0FB01EA59FE4F0081C0E0D0E09E
:1003400010E030E0F1E78F2EF1E09F2E860E971E31
:10035000ECE7AE2EE1E0BE2EA60EB71E90E0AC019B
:10036000440F551F480F591F440F551F440F551F69
:100370004C5B5D4F91E0C92ED12CE12CF12C3FC09C
:10038000F4012081632F70E0CB01820F911D803139
:10039000910524F02051230F12E007C0089724F0A4
:1003A0002850230F11E001C0230FF5018081FA01CD
:1003B000E10FF11DE80FF11D808190E002C09595DD
:1003C00087952A95E2F780FF0CC0D701C60104C0CB
:1003D000880F991FAA1FBB1F6A95D2F7C82BD92B6C
:1003E0000DC0D701C60104C0880F991FAA1FBB1FEB
:1003F0006A95D2F780959095C823D9233F5F30172F
:1004000008F4BECFCE01DF91CF911F910F91FF90E5
:10041000EF90DF90CF90BF90AF909F908F90089516
:100420008F929F92AF92BF92CF92DF92EF92FF9204
:100430000F931F93CF93DF934A0170E0FB01EA59BA
:10044000FE4F008110E030E041E7A42E41E0B42EE1
:10045000A60EB71E90E0EB01C458DE4FAC01440F6E
:10046000551F480F591F440F551F440F551FA1E03A
:10047000CA2ED12CE12CF12C4AC0F5012081632F2A
:1004800070E0CB01820F911D8031910524F0205145
:10049000230F12E007C0089724F02850230F11E023
:1004A00001C0230FC40102C0959587956A95E2F7B4
:1004B000612F70E080FF15C08881FB01E80FF11DFE
:1004C000E40FF51FEC5BFD4FD701C60104C0880F98
:1004D000991FAA1FBB1F2A95D2F72081282B2083A2
:1004E00015C08881FB01E80FF11DE40FF51FEC5BDF
:1004F000FD4FD701C60104C0880F991FAA1FBB1F5B
:100500002A95D2F780952081822380833F5F301720
:1005100008F4B3CFDF91CF911F910F91FF90EF902F
:10052000DF90CF90BF90AF909F908F9008950F93E2
:100530001F93CF93DF93082FCDE3D1E010E0FE01AE
:1005400045915491802F612F0E9410021F5F2296C7
:100550001B30A9F7DF91CF911F910F9108951F9341
:1005600010E0812F0E9497021F5F1630D1F71F9174
:100570000895582F30919102332351F1E6E9F2E0CA
:1005800040E090E007C08081851711F4292F41E0F9
:100590009F5F31969317B8F3442349F480E00895A0
:1005A000E22FF0E0EA56FD4F818180832F5F231711
:1005B000B8F3832F8150809391029FEF06C0E82FFC
:1005C000F0E0EA56FD4F90838F5F8031C0F301C0A9
:1005D000089581E00895EF92FF920F931F9330E00A
:1005E00040E050E0682F70E0E1E0EE2EF12C012DAC
:1005F000112DCB01042E02C0959587950A94E2F740
:1006000080FF0CC0D801C701042E04C0880F991FB9
:10061000AA1FBB1F0A94D2F7382B0CC0D801C70100
:10062000042E04C0880F991FAA1FBB1F0A94D2F77B
:10063000809538234F5F5F4F44305105D1F630939A
:10064000B90254E0759567955A95E1F7693021F440
:1006500081E08093B40214C0683031F41092B40287
:1006600081E08093B5020EC06B3041F41092B40269
:100670001092B50281E08093B60206C01092B402D7
:100680001092B5021092B60281E0809342011F9150
:100690000F91FF90EF900895883F10F480E0089547
:1006A000883F51F480918F0290919002019690932F
:1006B000900280938F0206C08A3F41F4109290020C
:1006C00010928F0281E080938C0208958C3F11F08C
:1006D00081E008951092900210928F0281E0809341
:1006E0008C020895EF92FF920F931F9320914D017A
:1006F00030914E0140914F0150915001D9019927FD
:10070000882782279327A427B5277C018D0125E020
:1007100016950795F794E7942A95D1F7E826F926D8
:100720000A271B278091510190915201A0915301FA
:10073000B091540180934D0190934E01A0934F01CD
:10074000B0935001209155013091560140915701CD
:10075000509158012093510130935201409353011D
:1007600050935401282739274A275B272E253F25F8
:1007700040275127EE0CFF1C001F111F2E253F257F
:10078000402751272093550130935601409357013C
:1007900050935801B901CA011F910F91FF90EF903A
:1007A0000895EF92FF920F931F937C010E947203B2
:1007B0009B01AC010027F7FC0095102F4070507092
:1007C000C801B7010E941A3E9B01AC019A0144275F
:1007D0005527C9011F910F91FF90EF9008958F92B7
:1007E0009F92AF92BF92CF92DF92EF92FF920F93C0
:1007F0001F93CF93DF93EA01EE2499249A9400E0AB
:1008000010E02FEF30E0FF24C62EDD2456010894BF
:10081000A108B108482F50E0BAE08B2E860E2BC0FD
:10082000FC01EE0FFF1FEC0FFD1F65917491461741
:10083000570700F1FC013196EE0FFF1FEC0FFD1F73
:10084000A591B491A417B507A8F09A2EE62E8C0DA9
:100850009D1DFC013196EE0FFF1FEC0FFD1F259132
:100860003491FC01EE0FFF1FEC0FFD1F8591949159
:10087000F82C8C01F3948F2D90E08A159B050CF4D5
:10088000CFCF8E2D90E0481B590B201B310B692DCB
:1008900070E0681B790B429FC001439F900D529FEF
:1008A000900D11240E94393E600F711FCB01DF9122
:1008B000CF911F910F91FF90EF90DF90CF90BF905D
:1008C000AF909F908F900895EF92FF920F931F9398
:1008D000282F80910F0390911003A0911103B091E4
:1008E00012038093EB029093EC02A093ED02B0937D
:1008F000EE0280912F03882309F451C00091EF028A
:100900001091F0020F5F1F4F1093F2020093F1025B
:10091000822F67E00E948D01081B190B1093F002D3
:100920000093EF0217FF04C01092F0021092EF0242
:10093000E0902603F09027030091280310912903EB
:100940006091F1027091F202882777FD8095982FCF
:10095000A80197010E941A3E6093EB027093EC028B
:100960008093ED029093EE026093C2027093C302F3
:100970008093C4029093C5026091EF027091F002DF
:10098000882777FD8095982F0E941A3E6093E70292
:100990007093E8028093E9029093EA027BC0822F71
:1009A00067E00E948D01AC019093F2028093F10206
:1009B00080914A01882389F0FA0106E0F595E795D0
:1009C0000A95E1F7EE0FFF1FE35EFE4F85919491CC
:1009D0009093F2028093F1024DC083E0483E5807A5
:1009E00044F52091EF023091F0022417350734F0DE
:1009F000265F3F4F3093F2022093F1026091F102A3
:100A00007091F202882777FD8095982F2091260318
:100A10003091270340912803509129030E941A3EE8
:100A20006093EB027093EC028093ED029093EE02E0
:100A300014C080910F0390911003A0911103B09105
:100A4000120380509240A040B0408093EB029093FC
:100A5000EC02A093ED02B093EE0280910A0388238A
:100A600049F08091EB029091EC02A091ED02B091DF
:100A7000EE0208C08091E7029091E802A091E9029D
:100A8000B091EA028093C2029093C302A093C40281
:100A9000B093C5021F910F91FF90EF900895EF92D0
:100AA000FF920F931F93CF93DF93AA2797FDA095F3
:100AB000BA2FBC01CD0124EA31E040E050E00E94B1
:100AC0001A3E2FEF33E040E050E00E94823E790171
:100AD0008A01309331032093300380914B018823A6
:100AE00089F0C9016AE070E00E944D3E70933103C5
:100AF00060933003FB01EE0FFF1FEF58FF4F45914E
:100B0000549128C0C9016AE070E00E944D3EDB01AB
:100B1000AA0FBB1F9D012D583F4FF901859194915C
:100B2000AF58BF4FFD01C591D4918C1B9D0B6AE05E
:100B300070E00E94393E9B01C7016AE070E00E94AC
:100B40004D3E289FA001299F500D389F500D112424
:100B50004C0F5D1FCA01DF91CF911F910F91FF9044
:100B6000EF90089568E00E948D018093AD02482FB8
:100B700050E09A013595279535952795217020935A
:100B8000F302817080934B019A01E4E0359527953B
:100B9000EA95E1F721702093F4029A0173E035950C
:100BA00027957A95E1F721705595479541704093C7
:100BB000AA02882311F41092AA0280918C02882341
:100BC00031F0222321F081E080934A0108951092B0
:100BD0004A010895CF93DF93682F592F2BE131E01D
:100BE00040E0C62FD52FF90185919491C817D907F8
:100BF00028F04F5F2E5F3F4F403199F7642F70E030
:100C0000660F771F9B01255E3E4FF90185919491F8
:100C1000675E7E4FFB0125913491821B930B62E04E
:100C200070E00E944D3E260F371FC217D30710F009
:100C3000E42F02C0E42FE150F0E0EE0FFF1FE55E6D
:100C4000FE4F25913491C901DF91CF9108950F9303
:100C50001F93CF93DF93082FC3E5D1E010E0FE018F
:100C6000859194910E94D103AC01802F612F0E9445
:100C700010021F5F2296183091F784E190E00E94E5
:100C8000D103AC01802F61E00E94100284E190E06A
:100C90000E94D103AC01802F62E00E941002DF911C
:100CA000CF911F910F9108951F93182F69E00E9413
:100CB0008D0180934301812F6AE00E948D01809312
:100CC00044011F91089589E18093B9011092BC01FC
:100CD0001092D4011092DF011092E2011092DE0115
:100CE0001092DD0183E991E09093DC018093DB01B8
:100CF0001092FE01109201021092FD011092FC016F
:100D00009093FB018093FA018AE192E00E945C2EAD
:100D100008958AE192E060E071E00E94972F0895C3
:100D2000BC018AE192E00E94972F8AE192E00E9442
:100D3000EF2FFBCF1F9310E08AE192E0612F40E09C
:100D40000E94DF2F1F5F1430B9F71F9108950F9392
:100D50001F930AE112E0C80163E540E00E947C2F86
:100D6000C80160E241E00E947C2FC801609143010C
:100D700042E00E947C2FC8016091440143E00E9440
:100D80007C2F1F910F91089589E192E00E94E63532
:100D90008EEF91E00E949123089583E080930303F6
:100DA0000E94C4060895282F8091BC029091BD0234
:100DB00001969093BD028093BC028617970764F05A
:100DC0001092BD021092BC0290E08091BE02882376
:100DD00009F491E09093BE028AE192E0622F409183
:100DE000BE020E94BB2E0895CF93DF93CCE5D1E0E5
:100DF0008AE192E0699140E00E94BB2E81E0C23618
:100E0000D807B1F78AE192E061E040E00E94BB2E92
:100E1000DF91CF9108950F931F938C0181E0809310
:100E20001E030E94753A60931F0370932003809302
:100E30002103909322038AE192E0B8010E94972F48
:100E40001F910F9108951F93182F85E091E00E9444
:100E50000B07A3E3B3E0212F30E0F901EE0FFF1FF2
:100E6000E20FF31FEE0FFF1FEE0FFF1FEC5BFD4FB6
:100E70008D91819383E0AF33B807D1F781E090E0A3
:100E8000A0E0B0E004C0880F991FAA1FBB1F2A95DD
:100E9000D2F780952091C10228232093C1028AE1D4
:100EA00092E00E94672E1F9108951F93182F8AE0E9
:100EB00091E00E940B078CE0189FD0011124AC5BDD
:100EC000BD4FE3E3F3E08D91819383E0EF33F807C7
:100ED000D1F71F9108951F93CF93DF93809125033E
:100EE0008823F1F0C0E0D0E0FE01E45AFE4F4091CB
:100EF000AD0250E00C2E02C0559547950A94E2F7DA
:100F000041708AE192E060810E94BB2E2196C5303B
:100F1000D10551F78AE192E067E040E00E94BB2EE4
:100F20008091A802823039F48AE192E06FE071E0AA
:100F30000E94972F39C080911E038823E9F00E94F8
:100F4000753A20911F033091200340912103509165
:100F50002203621B730B840B950B61547640804017
:100F6000904010F110921E030E94A7060E949A065C
:100F700085E08093230318C080915605813081F06D
:100F80008091BA02882361F410E08AE192E066E27F
:100F900070E0412F0E942C2F1F5F1430B1F702C068
:100FA0000E94A7060E949A06DF91CF911F91089593
:100FB000EF92FF920F931F938091E3029091E402CE
:100FC000A091E502B091E6022091F7023091F8027B
:100FD0004091F9025091FA02280F391F4A1F5B1FF6
:100FE0002093F7023093F8024093F9025093FA02EB
:100FF000E090EB02F090EC020091ED021091EE0215
:10100000B7FD16C02E153F054007510758F18091D6
:10101000E7029091E802A091E902B091EA02809380
:10102000F7029093F802A093F902B093FA021AC063
:101030002E153F054007510768F48091E702909113
:10104000E802A091E902B091EA0282179307A4078F
:10105000B50740F0E092F702F092F8020093F9022F
:101060001093FA0281E0809355054091F702509168
:10107000F8026091F9027091FA0289E192E00E940F
:101080000234109255051F910F91FF90EF90089533
:1010900080918D0290918E02892B09F45DC0209180
:1010A0006B0530916C0540916D0550916E058091F6
:1010B000170390911803A0911903B0911A03009798
:1010C000A105B10541F42093F7023093F802409353
:1010D000F9025093FA0280914A018823B1F060919D
:1010E0008F027091900280E090E02091DF023091B9
:1010F000E0024091E1025091E2020E94823E6115BD
:1011000071058105910541F525C00E94753A209130
:101110000B0330910C0340910D0350910E03621BA1
:10112000730B840B950B2091DF023091E00240910C
:10113000E1025091E202621773078407950760F09D
:101140000E94753A60930B0370930C0380930D0318
:1011500090930E030E94D80780918D0290918E0289
:10116000AA2797FDA095BA2F809317039093180391
:10117000A0931903B0931A0308950F931F93CF936D
:10118000DF938C01EC0197FF04C0CC27DD27C81B3F
:10119000D90B8AE192E0BE010E94B42FCE018D5995
:1011A0009F4F873C910538F48AE192E064E270E059
:1011B00041E00E942C2FCE0164E670E00E944D3E7B
:1011C0000996439750F4C436D1053CF48AE192E085
:1011D00064E270E042E00E942C2F17FF18C0C43672
:1011E000D10544F08AE192E065E270E040E00E94BF
:1011F0002C2F0DC02A972CF08AE192E065E270E076
:1012000014C08AE192E065E270E042E00FC0C85E7F
:10121000D34074F08AE192E061E070E040E00E9427
:101220002C2F8AE192E060E070E041E00E942C2FD8
:10123000DF91CF911F910F9108953F924F925F924E
:101240006F927F928F929F92AF92BF92CF92DF92D6
:10125000EF92FF920F931F93CF93DF93309032035F
:1012600052E6652E51E0752E4301CC244AE0442E0F
:10127000512CD090F602DD0CDD0CDC0C832D6D2D95
:101280000E948D018C018AE192E06C2D0E94A02EBB
:101290005C018AE192E06C2D0E94A92E7C018AE11A
:1012A00092E06C2D0E945D2ECD2DD0E0882309F4B4
:1012B00050C08AE192E0F401608140E00E94BB2EC0
:1012C000CA59DE4F8881282F30E08B3090F4C2015C
:1012D000821B930B9501082E02C0359527950A9421
:1012E000E2F7A70102C0559547958A95E2F7CA0132
:1012F00010C0C9010A979501082E02C0220F331FA2
:101300000A94E2F7F70102C0EE0FFF1F8A95E2F799
:10131000CF01281739074CF0201731070CF41AC1F8
:10132000081719070CF416C108C0021713070CF4AC
:1013300011C1801791070CF40DC18AE192E06C2D68
:101340000E948F2E8AE192E06C2DA5010E94B22EA0
:10135000E7C08AE192E0F401608141E00E94BB2E87
:10136000CA59DE4FF8804F2D50E0FAE0FF1550F0DB
:10137000C201841B950BE50102C0D595C7958A95DE
:10138000E2F708C04A505040E50102C0CC0FDD1F13
:101390004A95E2F7832D6D2DAE010E94100248E0C0
:1013A0004F1578F498012C1B3D0B37FF03C0309587
:1013B00021953F4F8091410190E082179307F4F40B
:1013C0000EC033E0159507953A95E1F7CE0123E07D
:1013D000959587952A95E1F70817190779F0C09236
:1013E000230381E080931E030E94753A60931F03DC
:1013F0007093200380932103909322038091230311
:101400008C1509F08DC0DD2079F480914B0140915D
:10141000300350913103882319F0EA01A49760C08A
:10142000EA01C856D1405CC054E0D516E9F4809179
:101430004A01882369F0FE01B3E0F595E795BA9576
:10144000E1F7EE0FFF1FE55EFE4F259134912EC0B0
:10145000C530D1050CF442C0CA30D1051CF4C1E03E
:10146000D0E03EC029973CC085E0D81661F4CE3666
:10147000D1051CF4CE56D04033C0C339D10574F128
:10148000C259D0402DC0E7E0DE1651F580914A01E7
:101490008823F9F0FE0176E0F595E7957A95E1F776
:1014A000EE0FFF1FE35EFE4F25913491C9010197B6
:1014B000479740F488E190E0B9010E944D3EEB016E
:1014C00011E00FC0C90168E170E00E944D3EEB01E0
:1014D00007C0C091F102D091F20202C0C0E0D0E09A
:1014E00010E08091F602E82FF0E0EE0FFF1FEE0F04
:1014F000FF1FEC0DF11DE859FF4F659174918AE1D2
:1015000092E040E00E947C2FCE010E94BD08112392
:1015100039F08AE192E067E270E041E00E942C2F0E
:10152000C3940894811C911CF4E0CF1609F0A1CE5D
:10153000809191028823D1F48AE192E0F3016191D4
:101540003F0140E00E94BB2EF6E66F16F1E07F06F9
:1015500099F70CC0C5018E199F0997FF03C090959C
:1015600081959F4F40970CF0E8CEECCEDF91CF9164
:101570001F910F91FF90EF90DF90CF90BF90AF90B1
:101580009F908F907F906F905F904F903F900895C5
:101590001F93982F80915605813009F0D6C0109185
:1015A0009402992321F0913009F0CFC057C08AE10D
:1015B00092E060E00E945D2E8823E1F4812F60E0DC
:1015C0000E948D010E944F059C019093AC02809374
:1015D000AB0280919302873020F080914B018823E9
:1015E00049F4A901662757FD6095762F89E192E0BD
:1015F0000E9436348AE192E061E00E945D2E8823E9
:1016000069F4812F61E00E948D01E3E0880F991F4A
:10161000EA95E1F79093700580936F058AE192E077
:1016200062E00E945D2E882341F4812F62E00E94D7
:101630008D019093AF028093AE028AE192E063E065
:101640000E945D2E882309F080C0812F63E00E94F4
:101650008D019093B1028093B00277C0812F64E036
:101660000E948D019C0190938E0280938D02809147
:101670004A01882369F0F90173E0F595E7957A95B9
:10168000E1F7EE0FFF1FE55EFE4F8591949107C0D5
:10169000822F880F68E043ED50E00E94EF03A0E046
:1016A000B0E08093DF029093E002A093E102B09358
:1016B000E2028AE192E061E00E945D2E8823B9F4A3
:1016C000812F65E00E948D016AE043EF50E00E94A7
:1016D000EF03A0E0B0E080589E43A040B04080936C
:1016E000E3029093E402A093E502B093E6028AE15C
:1016F00092E062E00E945D2E882321F580912F0305
:10170000882301F5812F66E00E948D019093F002FD
:101710008093EF02AA2797FDA095BA2F2091260368
:10172000309127034091280350912903BC01CD013A
:101730000E941A3E6093E7027093E8028093E902E8
:101740009093EA02812F0E9464041F9108950F93E1
:101750001F93982F10922F032091110230911202A3
:10176000409113025091140220930F033093100301
:10177000409311035093120380914B01882329F564
:10178000973118F19A3408F5892F90E04797909394
:10179000F0028093EF0200919402CA01B9012CE398
:1017A00030E040E050E00E94603E209326033093FA
:1017B0002703409328035093290380910A03882329
:1017C000B1F181E080932F0332C0192F1751E091BE
:1017D0009402CA01B9012AE0969587957795679595
:1017E0002A95D1F71B3290F40E2F60932603709345
:1017F000270380932803909329038E2F66E00E948D
:101800008D019093F0028093EF0212C00E2F60932F
:1018100026037093270380932803909329038E2F28
:1018200066E00E948D019093F0028093EF021FEF1B
:101830006091EF027091F002882777FD8095982FD4
:1018400020912603309127034091280350912903CA
:101850000E941A3E6093E7027093E8028093E902C7
:101860009093EA02802F0E94B205802F62E00E94CE
:101870008D019093AF028093AE02802F63E00E94AF
:101880008D019093B1028093B00281E08093550561
:101890001F3F49F0E12FF0E0EE0FFF1FEF58FF4F21
:1018A0008591949106C0802F60E00E948D010E9476
:1018B0004F059093AC028093AB024091AB025091E4
:1018C000AC02662757FD6095762F89E192E00E9471
:1018D0003634802F61E00E948D01880F8093410291
:1018E00090E0880F991F880F991F9093700580933F
:1018F0006F05802F64E00E948D019C0190938E0201
:1019000080938D0280914A01882369F0F901B3E048
:10191000F595E795BA95E1F7EE0FFF1FE55EFE4FEF
:101920008591949107C0822F880F68E043ED50E0C5
:101930000E94EF03A0E0B0E08093DF029093E0020A
:10194000A093E102B093E202802F65E00E948D0136
:101950006AE043EF50E00E94EF03A0E0B0E080585F
:101960009E43A040B0408093E3029093E402A09392
:10197000E502B093E602B7FF0AC080918D02909114
:101980008E02892B21F081E080930A0302C010921D
:101990000A03802F0E9464040E94753A60930B032F
:1019A00070930C0380930D0390930E034091C20239
:1019B0005091C3026091C4027091C50289E192E026
:1019C0000E9402348091C2029091C302A091C4028D
:1019D000B091C5028093F7029093F802A093F902A8
:1019E000B093FA02109255051F910F910895EF924E
:1019F000FF920F931F93E0906B05F0906C050091A0
:101A00006D0510916E058091A802823009F045C0E5
:101A100080914A01882371F060911303709114033F
:101A200080918F02909190020E94393E892B09F09B
:101A3000DDC019C080910A032091FF02309100039C
:101A40004091010350910203882339F02E153F0580
:101A50004007510708F4CAC006C0E216F30604079F
:101A6000150708F4C3C081E0809355054091FB023F
:101A70005091FC026091FD027091FE0289E192E0BA
:101A80000E940234109255058091FB029091FC0255
:101A9000A091FD02B091FE029EC080910A03909138
:101AA0004A01882309F450C0992399F06091F1020A
:101AB0007091F20283E0683E780709F497C0809144
:101AC0008F02909190020E94393E892B09F457C0F1
:101AD0008DC08091E7029091E802A091E902B09157
:101AE000EA028E159F05A007B107C8F08091F302A6
:101AF000882399F08091EB029091EC02A091ED0285
:101B0000B091EE028093F7029093F802A093F9024D
:101B1000B093FA020E94D80702C00E94C4068091C6
:101B20000F0390911003A0911103B09112038855F7
:101B30009240A040B040E816F9060A071B0708F4D7
:101B400055C00E94D80752C0992329F16091F10233
:101B50007091F20283E0683E780709F447C0209153
:101B60008F0230919002C9010E94393E892BF1F514
:101B7000809115039091160328173907B9F18091C8
:101B8000F302882389F181E08093550580919302C7
:101B90000E94A70B2BC08091EB029091EC02A091C8
:101BA000ED02B091EE02E816F9060A071B07F0F005
:101BB0008091F3028823C1F081E0809355058091E4
:101BC00093020E94A70B8091C2029091C302A09140
:101BD000C402B091C5028093F7029093F802A093DB
:101BE000F902B093FA0202C00E94C40680918F02EB
:101BF0009091900290931603809315031F910F917B
:101C0000FF90EF90089580910303813009F471C033
:101C1000813038F0823009F475C0833009F0E0C0BB
:101C2000DDC080911C0390911D03892BB1F480913C
:101C30000A03882339F081E090E090931D0380939C
:101C40001C03089581E0809303031092090310920E
:101C5000080389E192E060E0BEC00E94753A2091DD
:101C60000403309105034091060350910703621B62
:101C7000730B840B950B20911C0330911D0344279B
:101C800037FD4095542F621773078407950708F4B2
:101C9000A7C00E94753A6093040370930503809374
:101CA00006039093070380911C0390911D032091DC
:101CB0000803309109034E971CF42350304002C0B2
:101CC00021503040309309032093080380911B0377
:101CD00090E02091080330910903821793070CF4D8
:101CE00076C0109209031092080381E080930303E9
:101CF0006EC060911B03609308031092090389E191
:101D000092E069C080915605813009F055C08091FC
:101D1000B0029091B102892B81F483E08093030398
:101D200084E290E0909309038093080389E192E0B4
:101D300064E20E94E7330E94C4060E94753A209133
:101D40000403309105034091060350910703621B81
:101D5000730B840B950B2091B0023091B102442794
:101D600037FD4095542F6217730784079507C0F11C
:101D70000E94753A609304037093050380930603F1
:101D8000909307038091B0029091B10220910803D3
:101D9000309109034E971CF42D5F3F4F02C02F5F17
:101DA0003F4F3093090320930803809108039091DB
:101DB0000903849764F006C084E290E090930903DD
:101DC0008093080383E0809303030E94C40689E1A3
:101DD00092E0609108030E94E73308950E94C406D0
:101DE00008950E94753A60930403709305038093ED
:101DF00006039093070380910303823031F089E159
:101E000092E0609108030E94E73382E0809303032D
:101E100008950F931F93CF93DF9380912503882319
:101E2000E1F58AE192E061E00E943E308823A9F169
:101E30008091F502882371F11092F5021FEFC0E046
:101E4000D0E0FE01E45AFE4F8AE192E060810E94F8
:101E50003430882329F080919602C81709F41C2F8A
:101E60002196C630D10569F71F3F19F010939302F0
:101E700014C0E6E9F2E08FEF819392E0E63AF907C9
:101E8000D9F710929102109293020E94F10E1092D3
:101E9000A80203C081E08093F5028AE192E061E04C
:101EA0004091F5020E94BB2EDF91CF911F910F91BF
:101EB0000895EF92FF921F93182F7B010E94753AAD
:101EC00060930403709305038093060390930703C4
:101ED00085E290E090930903809308031092030336
:101EE00089E192E065E20E94E733169516958FE14D
:101EF000811B80931B03F0921D03E0921C031F9132
:101F0000FF90EF900895CF93DF93AC01C62FD0E000
:101F10008091C10290E0062E02C0959587950A94A3
:101F2000E2F780FF12C0CC0FDD1FCC0FDD1FCA53BC
:101F3000DD4F488159818EEF91E06FED71E021E036
:101F40000E941E258823B9F544C08EEF91E06FED05
:101F500071E021E00E945B288823D9F1FE01EE0F99
:101F6000FF1FEE0FFF1FEA53FD4F8091EA01909192
:101F7000EB01A091EC01B091ED0135E0B695A7958C
:101F8000979587953A95D1F70197A109B109808373
:101F90009183A283B38381E090E0A0E0B0E004C02D
:101FA000880F991FAA1FBB1FCA95D2F72091C102A3
:101FB000282B2093C10289E192E06EEF71E00E942C
:101FC0006937882311F081E005C08EEF91E00E940F
:101FD000912380E0DF91CF9108950F931F9390910B
:101FE0004401892F8150809344018033B4F48AE501
:101FF00080934401809143018150809343018B532E
:10200000863018F48AE38093430180914301803342
:10201000DCF58AE58093430104C09C539630A0F51B
:102020008AE38093440130C08AE192E00E94EF2F5E
:102030000E94890680914C0190914401981B9093D5
:1020400044018F5F80934C019033ACF410934401B2
:10205000809143018150809343018B53863010F46B
:102060000093430180914301803354F41093430162
:102070001093440105C09B53963040F400934401F3
:1020800081E080934C0102C00AE31AE58EEF91E0F3
:102090006FED71E043E451E021E00E945B2888236A
:1020A00019F28EEF91E00E9491236091940281E0F9
:1020B00090E0A0E0B0E0062E04C0880F991FAA1F90
:1020C000BB1F0A94D2F780952091C1022823209348
:1020D000C10283E491E00E94830F882311F40E94DF
:1020E000ED0F0E94C40681E080934C011F910F9177
:1020F00008950F931F9380914401982F9F5F9093B1
:1021000044018953873020F481E4809344014BC01B
:102110009B350CF448C020E3209344018091430197
:10212000982F9F5F909343018953873020F481E477
:102130008093430138C09B35B4F120934301209331
:10214000440131C08AE192E00E94EF2F0E9489068B
:1021500080914C0190914401980F909344018F5FBE
:1021600080934C01892F8A53873018F400934401DF
:1021700016C09B35D4F01093440180914301982FF1
:102180009F5F909343018953873018F40093430174
:1021900006C09B3524F0109343011093440181E065
:1021A00080934C0102C010E301E48EEF91E06FEDEB
:1021B00071E043E451E021E00E945B28882311F2A2
:1021C0008EEF91E00E9491236091940281E090E073
:1021D000A0E0B0E0062E04C0880F991FAA1FBB1F05
:1021E0000A94D2F780952091C10228232093C1023E
:1021F00083E491E00E94830F882311F40E947910F8
:102200000E94C40681E080934C011F910F910895B4
:102210001F93182F0E94C40683E491E0612F0E944F
:10222000830F85E0809323030E94A7061F910895E2
:102230001F93182F8093930287518D3390F48091D0
:1022400094020E945406809194020E940811812FEA
:102250000E94A70B6091AE027091AF028091A6021E
:1022600014C01630A0F410939402812F0E945406DB
:10227000809194020E940811809194020E94A70B01
:102280006091AE027091AF028FE70E94590F1F91CB
:10229000089580912403882309F071C18AE192E0B6
:1022A0006AE00E943E30882309F43FC00E94C406C1
:1022B0000E94791040914301552747FD5095809128
:1022C000940269E00E94100240914401552747FDA5
:1022D0005095809194026AE00E94100290919402BD
:1022E0009093930280919102882321F0892F0E947C
:1022F00018110FC00E94A70681E080931E030E9460
:10230000753A60931F037093200380932103909389
:1023100022030E94753A60932A0370932B038093E3
:102320002C0390932D0310922E038AE192E069E032
:102330000E943E30882309F43FC00E94C4060E94D8
:10234000ED0F40914301552747FD50958091940230
:1023500069E00E94100240914401552747FD5095C5
:10236000809194026AE00E941002909194029093EE
:10237000930280919102882321F0892F0E941811E5
:102380000FC00E94A70681E080931E030E94753A49
:1023900060931F0370932003809321039093220383
:1023A0000E94753A60932A0370932B0380932C0349
:1023B00090932D0310922E038AE192E069E00E942F
:1023C0003430882341F48AE192E06AE00E9434309C
:1023D000882309F495C080912E03882311F50E946B
:1023E000753A20912A0330912B0340912C03509190
:1023F0002D03621B730B840B950B69557240804053
:10240000904008F47DC081E080932E030E94753ACD
:1024100060932A0370932B0380932C0390932D03D6
:102420006FC00E94753A20912A0330912B0340918E
:102430002C0350912D03621B730B840B950B615978
:1024400071408040904008F45BC00E94753A6093F0
:102450002A0370932B0380932C0390932D038AE11E
:1024600092E069E00E943430882389F08091430132
:102470008150809343018B53863018F48AE3809314
:102480004301809143018033ECF48AE517C08AE16F
:1024900092E06AE00E943430882391F180914301F8
:1024A000982F9F5F909343018953873020F481E4F4
:1024B0008093430107C09B352CF080E38093430158
:1024C0008093440140914301552747FD50958091E9
:1024D000940269E00E9410028AE192E06091430157
:1024E00042E00E947C2F81E080931E030E94753A97
:1024F00060931F0370932003809321039093220322
:102500008AE192E06AE00E944830882339F48AE147
:1025100092E069E00E944830882389F180912E037F
:10252000882369F1309194023093930281E090E026
:10253000A0E0B0E0032E04C0880F991FAA1FBB1FA4
:102540000A94D2F780952091C10228232093C102DA
:1025500080919102882321F0832F0E941811089501
:102560000E94A70681E080931E030E94753A609343
:102570001F037093200380932103909322030895F7
:102580008091E3029091E402A091E502B091E6020D
:10259000B7FF0AC080918D0290918E02892B21F0A5
:1025A00081E080930A0302C010920A038091F40232
:1025B0008823E9F082E090E00E94D103892BB9F4EE
:1025C0008091E3029091E402A091E502B091E602CD
:1025D000B095A095909581959F4FAF4FBF4F809339
:1025E000E3029093E402A093E502B093E6028091A7
:1025F0009102882341F480910303823021F080917D
:10260000A902882359F180915505882339F40E9445
:10261000030E0E94F70C0E94480820C0809194028B
:102620000E94B2058091F3028823B1F080910A03E1
:10263000882369F089E192E00E94E63589E192E021
:102640006EEF71E00E9469370E94D80707C0809141
:1026500093020E94A70B02C00E94C40680919102BF
:10266000882329F1809194020E94B2058091560539
:10267000813021F4809155058823C9F08091F302BF
:102680008823A9F080910A03882369F089E192E008
:102690000E94E63589E192E06EEF71E00E946937B1
:1026A0000E94D8070895809196020E9418110895FB
:1026B0001F93182F863020F48AE192E00E94672E43
:1026C000812F0E94B9028823C1F180919102882351
:1026D00049F19091960280919302981759F1809157
:1026E000AA028823D9F09731C8F09234B8F49093B5
:1026F0009302E92FF0E0EE0FFF1FED5BFF4F4591D6
:1027000054915093AC024093AB02662757FD6095FD
:10271000762F89E192E00E9436340CC0892F0E9406
:10272000181106C08091A902882321F40E94F10E9D
:102730001092A8028091960200C01F9108951F93E5
:10274000182F863020F48AE192E00E94672E809153
:1027500091028F3021F48091A5020E94B902812F4D
:102760000E94B902209191022031B0F4222351F04D
:10277000922FE92FF0E0EA56FD4F82913196808347
:102780009150B9F7109396022F5F2093910281E048
:10279000809392021092A70280919202882339F1CD
:1027A0008091AA028823F9F01731E8F01234D8F4A6
:1027B000809191028230B8F010939302E12FF0E003
:1027C000EE0FFF1FED5BFF4F459154915093AC020C
:1027D0004093AB02662757FD6095762F89E192E022
:1027E0000E94363404C0809196020E9418111F91F5
:1027F00008950F931F93CF93DF93CCE5D1E010E0C2
:102800008091F5028823B9F08AE192E068810E9404
:102810003E30882379F1809193020E9458131093DF
:10282000930210939402812F0E949F138091930230
:10283000809332031FC008818AE192E0602F0E94DA
:102840003E30882359F01093930210939402812F05
:102850000E949F1380919302809332038AE192E059
:10286000602F0E944830882329F0812F0E9458133E
:102870008093930280919402811769F48091910270
:10288000882349F0E12FF0E0E45AFE4F8AE192E01C
:10289000608141E004C08AE192E0688140E00E94EA
:1028A000BB2E1F5F2196163009F0AACFDF91CF9182
:1028B0001F910F9108951F93982F162F80919502C5
:1028C000481759F4892F8150662319F40E94581330
:1028D00004C00E949F131093A6021F91089588EBD5
:1028E00091E060E04AE00E94BA1E882321F484E16E
:1028F00091E00E9490068DEB91E068EB71E041E081
:102900000E94682A882339F48DEB91E068EB71E02E
:1029100040E00E94682A8FED91E06DEB71E00E942B
:10292000482008950F931F93CF93DF9382E897E099
:102930006FEF73E00E941A3A80939502813148F05C
:1029400082E897E06FEF73E040E00E94213A109236
:1029500095028AE192E00E94BE318AE192E068E04D
:102960000E943430882339F082E897E06BEF73E0FF
:1029700040E00E94213A8AE192E062E00E94343015
:10298000882339F082E897E06BEF73E044E00E941F
:10299000213A8AE192E061E00E943430882339F0E4
:1029A00082E897E06BEF73E049E00E94213A82E809
:1029B00097E06BEF73E00E941A3A8D5F80934101BC
:1029C0008C3039F0873029F0833019F083E0809320
:1029D0004101C0E0D0E006E0FE01E45AFE4F8AE18A
:1029E00092E060810E943430882391F08AE192E085
:1029F0006BE00E943430809FC00111244C2F480F9F
:102A00004093950282E897E06FEF73E00E94213ACD
:102A10002196C630D10501F78091950290E001968C
:102A20000E94BD088AE192E063E440E00E947C2FAE
:102A30008AE192E068E441E00E947C2F8AE192E022
:102A400061E041E00E94DF2F80915605813049F41A
:102A500004C08AE192E00E94BE318091550588232E
:102A6000C1F30E94C406DF91CF911F910F91089589
:102A7000E6E9F2E08FEF819392E0E63AF907D9F7C1
:102A8000109291020E94921484E198E042E15AE788
:102A900060E070E00E945A3C0895EF92FF920F931D
:102AA0001F93CF93DF93082F162F0E94CD061F5C34
:102AB00010933B01005D00933A018EEF91E06FEDC2
:102AC00071E049E351E022E40E945B28882339F158
:102AD000EE24FF2411C08AEF91E069910E949329AE
:102AE0000F5F1F4F0C301105B1F70894E11CF11C6A
:102AF00086E0E816F10471F0E701CC0FDD1FCE0D82
:102B0000DF1DCC0FDD1FCC0FDD1FCC5BDD4F00E0E8
:102B100010E0E1CF8EEF91E00E94912381E0DF9100
:102B2000CF911F910F91FF90EF9008950F931F93F6
:102B300080914302609142020E944D1502E817E025
:102B4000C80169EE73E0409143020E94213AC80136
:102B50006AEE73E0409142020E94213AC80168EE99
:102B600073E041E00E94213A0C9400001F910F9104
:102B70000895FF920F931F93CF93DF93F82E0E9437
:102B8000C40680914302805D80934301809142029C
:102B900026E0829FC00111248F0D8A3010F4805DE1
:102BA00001C0895C809344018EEF91E06FED71E08C
:102BB00043E451E021E00E945B28882369F08EEF16
:102BC00091E00E9491238FED91E063E471E00E9417
:102BD0002329882309F4F2C08EEF91E06FED71E0B4
:102BE00043E451E000E010E020E436E00E944B298D
:102BF000882309F4E3C089E192E062E276E540E0EF
:102C000020E40E94D7338AE192E069E171E00E94FA
:102C1000972FCF2DD0E0FE01E45AFE4F10818AE1BC
:102C200092E0612F41E00E94BB2E8091DE028F5F17
:102C30008093DE02843030F01092DE028AE192E06E
:102C40000E94EF2F8AE192E00E9452308AE192E0E6
:102C50000E94EF2F82E062E370E00E94D3068AE1D7
:102C600092E061E00E943E30882399F090E08091EC
:102C7000C002882309F491E09093C002892F91113A
:102C800081E080937105529A539A549A5A9A559AB0
:102C90005D988AE192E061E04091C0020E94BB2E03
:102CA0008AE192E062E00E943E308823C9F48AE122
:102CB00092E068E00E943E30882309F4B6CF10927B
:102CC000BB021092BF028EEF91E00E949B238EEF19
:102CD00091E00E9491231092BA0287E880937A00D3
:102CE0008091BA02882309F467C01092BB02109247
:102CF000BF021092BA0289E192E06EEF71E042E207
:102D000056E520E000E40E940136882329F48EEF86
:102D100091E00E949B2352C08AE192E0612F0E94C1
:102D20001A3086E062E00E94EA3A86E00E947D3B2B
:102D3000892BD9F309C086E00E947D3B892B21F4C1
:102D400089E192E00E94E63580915605823099F340
:102D500089E192E00E94E63589E192E06EEF71E050
:102D60000E944F348EEF91E00E9491238F2D0E949C
:102D7000970240914301552747FD50958F2D69E0FB
:102D80000E94100240914401552747FD50958F2D18
:102D90006AE00E94100281E090E0A0E0B0E004C090
:102DA000880F991FAA1FBB1FCA95D2F78095209143
:102DB000C10228232093C1020E949615DF91CF9172
:102DC0001F910F91FF900895CF93DF938091BF02E1
:102DD000882309F04EC08AE192E062E00E943E3012
:102DE000882339F48AE192E068E00E943E3088232B
:102DF00041F01092BA0287E880937A0081E08093D4
:102E000024038AE192E061E00E943E30882399F039
:102E100090E08091C002882309F491E09093C00271
:102E2000892F911181E080937105529A539A549A97
:102E30005A9A559A5D988AE192E061E04091C00209
:102E40000E94BB2EC0E0D0E0FE01E45AFE4F8AE1B2
:102E500092E060810E943E30882339F0C093BF0227
:102E60008C2F609142020E94B9152196C630D1057F
:102E700059F7DF91CF910895EF92FF920F931F932F
:102E8000CF93DF93182F062F663008F005E0183C2B
:102E900010F010E003C0193008F019E00F5C009347
:102EA0003B010153105D10933A011053009342020D
:102EB000109343020E94CD06E6E9F2E08FEF819382
:102EC00092E0E63AF907D9F7109291028EEF91E07D
:102ED0006FED71E049E351E021E00E945B28882317
:102EE00079F40E94AF02812F602F0E944D158EEF62
:102EF00091E06FED71E049E351E021E00E945B2831
:102F0000EE24FF2411C08EEF91E00E94CA24899321
:102F10000F5F1F4F0C301105B1F70894E11CF11C35
:102F200086E0E816F10471F0E701CC0FDD1FCE0D4D
:102F3000DF1DCC0FDD1FCC0FDD1FCC5BDD4F00E0B4
:102F400010E0E1CF8EEF91E00E9491238AE192E0C0
:102F50000E94672E8EE191E00E940B078AE192E0C9
:102F600060913B0143E00E947C2F8AE192E06091F6
:102F70003A0142E00E947C2F1092C102DF91CF9172
:102F80001F910F91FF90EF9008951F93462F81306E
:102F900061F48091940261E050E00E9410028AE1A5
:102FA00092E00E948A2E80E061C08034B1F4862FC6
:102FB00090E026E0959587952A95E1F78093A90200
:102FC000882309F059C080919102882309F054C0E8
:102FD0000E94F10E1092A8024FC08823C1F470E045
:102FE00080E090E026E030E040E050E00E941A3EB1
:102FF0009B01AC0117E055954795379527951A9594
:10300000D1F780914302622F0E943C1735C0182FE0
:103010001656183088F52091940270E0E12FF0E008
:10302000EA59FE4F8081482F50E0883058F487E0FD
:1030300090E0841B950BAB0102C0559547958A958E
:10304000E2F709C047505040CB0102C0880F991FDA
:103050004A95E2F7AC01822F612F0E9410028AE1AB
:1030600092E00E948A2E812F869586950E94C80A3A
:103070008AE192E00E94672E1F910895982F809117
:103080009502481719F4892F0E94C51708951F93B8
:10309000182F0E944C03882309F041C017FF04C079
:1030A000812F0E94EB023BC0809142019091B602B9
:1030B000882399F010924201992341F48091B4023F
:1030C000882321F48091B502882319F01093B70268
:1030D00026C081E08093420122C01093B80281E0B3
:1030E00080934201992341F08091B702612F409172
:1030F000B9020E943E1813C08091B402882321F0C7
:103100008091B702612F07C08091B502882339F002
:103110008091B70260E04091B9020E945B141F9158
:10312000089519C084E198E00E94E13C9093B302B5
:103130008093B20218161906ACF4803491052CF075
:1031400084E198E00E943B3D06C084E198E00E9443
:10315000123D0E94471884E198E00E94E13C181655
:10316000190604F3089580914302609142020E947F
:103170003C170895CF92DF92EF92FF920F931F9327
:10318000CF93DF938AE192E068E00E943430082F09
:10319000CCE5D1E010E0FF24F394002371F08AE144
:1031A00092E068810E943E30882339F0F092240337
:1031B00080914302612F0E943C171F5F21961630B9
:1031C00061F7002389F08AE192E06AE00E943E30D4
:1031D000882351F081E080932403809143028F5F24
:1031E000609142020E943C178AE192E068E00E94EE
:1031F0003430882389F08AE192E069E00E943E3011
:10320000882351F081E08093240380914302815010
:10321000609142020E943C178AE192E068E00E94BD
:1032200034308823C9F08AE192E062E00E943E30A7
:10323000882391F081E08093240380914302609180
:1032400042020E944D15882319F083E291E002C0EA
:1032500088E291E00E940B078AE192E06BE00E9415
:10326000343080932503882309F462C18AE192E017
:1032700068E00E943430882309F05AC18AE192E064
:103280006AE00E943E30882339F081E08093240375
:10329000809194020E9455078AE192E069E00E94C1
:1032A0003E30882339F081E080932403809194029A
:1032B0000E9423078AE192E062E00E943E30882368
:1032C00009F454C08091A8028230F1F581E0809326
:1032D00024036091FB027091FC028091FD029091A9
:1032E000FE0220912603309127034091280350913C
:1032F00029030E94603E8091940266E0A9010E9429
:1033000010026091FF02709100038091010390917F
:103310000203209126033091270340912803509106
:1033200029030E94603E8091940267E0A9010E94F7
:1033300010021092A8028AE192E00E94672E80910A
:1033400094020E94A70B12C081E080932403809115
:103350004302609142020E944D15882319F083E2D6
:1033600091E002C088E291E00E940B07C0E0D0E04B
:1033700001E031E0C32ED12CE12CF12CFE01E45A06
:10338000FE4F8AE192E060810E943E308823C9F1BD
:10339000009324038091940268E00E948D01282FFD
:1033A00090E00C2E02C0959587950A94E2F780FD77
:1033B0000EC0D701C6010C2E04C0880F991FAA1F8A
:1033C000BB1F0A94D2F7282B2093AD020EC0D70161
:1033D000C6010C2E04C0880F991FAA1FBB1F0A9498
:1033E000D2F7809582238093AD024091AD02809107
:1033F000940268E050E00E941002809194020E94C2
:10340000B2052196C530D10509F0B8CF8AE192E026
:1034100061E00E943E30882309F478C08091A802C0
:103420008F5F8093A802833010F01092A8028091E1
:10343000A8028130F1F480916B0590916C05A09108
:103440006D05B0916E058093FB029093FC02A093F2
:10345000FD02B093FE0280914A01882309F456C010
:1034600080918F02909190029093140380931303A4
:103470004DC0823009F04AC080914A018823A9F0EA
:1034800080918F0290919002209113033091140348
:10349000821B930B90931403809313030E94EA05FD
:1034A000909314038093130310C080916B05909147
:1034B0006C05A0916D05B0916E058093FF0290930D
:1034C0000003A0930103B093020381E080935505AC
:1034D0004091FB025091FC026091FD027091FE024E
:1034E00089E192E00E940234109255058091FB021E
:1034F0009091FC02A091FD02B091FE028093F70230
:103500009093F802A093F902B093FA028AE192E054
:1035100067E00E943E30882359F081E080932403C5
:10352000809194020E942706809194020E94A70B2A
:1035300080912403882379F000E010E08AE192E092
:10354000612F0E943430080F1F5F1031B9F700233C
:1035500011F410922403DF91CF911F910F91FF90EE
:10356000EF90DF90CF9008958091BA028823D1F038
:103570008AE192E061E00E94012F8AE192E00E94DC
:10358000EF2F8AE192E00E9452308AE192E06DE2F0
:1035900071E00E94972F0E94E4168AE192E00E9457
:1035A000EF2F08958AE192E00E9452308AE192E082
:1035B0000E94EF2F8AE192E00E9498310E94BA188F
:1035C0000E94090F809124038823C1F58AE192E0CB
:1035D00068E00E944830882369F08091F6028F5F8E
:1035E0008093F602823010F01092F6028AE192E0A7
:1035F0000E94672E8AE192E062E00E9448308823B0
:10360000D9F00E94CD061092F5020E94F406E6E978
:10361000F2E08FEF819392E0E63AF907D9F7109242
:10362000910281E08093BA0289E192E062E276E55C
:1036300040E020E40E94D7330E94F9138AE192E02F
:1036400062E040E00E94BB2E6091F6026E5F8AE16C
:1036500092E00E94012F0E9449118091F6020E947F
:10366000C80A0E941D090E946B0708950E949118C4
:103670000E9491180E94B41A0E9491180E949118F9
:103680000E94C0120E9491180E94911808958AE128
:1036900092E00E94CC310E946F1482E897E068EEBD
:1036A00073E00E941A3A882381F482E391E067E094
:1036B0000E94830F89E192E042E256E560E070E00B
:1036C0000E9436341092550517C082E897E068EEE4
:1036D00073E040E00E94213A82E897E06AEE73E0EE
:1036E0000E941A3A8093420282E897E069EE73E002
:1036F0000E941A3A809343020E9438150E94B31820
:1037000087E880937A0008958091C10085FDFCCF01
:103710008091C00085FFF8CF6093C60081E090E003
:10372000089510924203109241038BE891E0909328
:10373000400380933F030895FF920F931F93CF930D
:10374000DF938B010E94753AEB01FF24FA9409C0C4
:103750000E94753A6C1B7D0B6017710710F080E0BA
:1037600008C0FEBC0DB407FEFDCF8EB58F3F81F7BC
:1037700081E0DF91CF911F910F91FF900895FC019F
:1037800022812D3010F046E002C0422F4695242FB2
:1037900030E0C9019595879580658CBD40FF02C0DA
:1037A00080E004C080E0463009F081E08DBD80817A
:1037B00060E00E94293B0895FF920F931F93DF93CF
:1037C000CF9300D000D0CDB7DEB78C01F62E298381
:1037D0003A834B835C830E94BF1BC8016CE271E09B
:1037E0000E949C1B8F2D80648EBD0DB407FEFDCF03
:1037F000FE0131969E012350304083818EBD0DB471
:1038000007FEFDCF3197E217F307B9F7FF2011F05C
:1038100087E801C085E98EBD0DB407FEFDCF8CE0C1
:10382000F81631F48FEF8EBD0DB407FEFDCF8EB5C7
:1038300090E02FEF2EBD0DB407FEFDCF8EB587FFB4
:1038400002C09150B9F7F80183830F900F900F9049
:103850000F90CF91DF911F910F91FF900895FC0180
:10386000808161E00E94293B8FEF8EBD0DB407FE81
:10387000FDCF0895CF93DF93EC010E94BF1BCE01D3
:1038800068E572E00E949C1B882389F08DEF8EBD55
:103890000DB407FEFDCFCE0168E572E00E949C1BCF
:1038A000882329F0CE010E942F1C81E006C082E10E
:1038B0008983CE010E942F1C80E0DF91CF91089573
:1038C000AF92BF92CF92DF92EF92FF920F931F932E
:1038D000CF93DF93EC015A016B017801890167E313
:1038E00020E030E040E050E00E94DC1BCE0167E1C8
:1038F000A80197010E94DC1B882311F089E013C006
:103900008C81833039F049E0AA0CBB1CCC1CDD1C37
:103910004A95D1F7CE0169E1A60195010E94DC1B11
:10392000882339F087E08983CE010E942F1C80E034
:1039300004C0CE010E942F1C81E0DF91CF911F9126
:103940000F91FF90EF90DF90CF90BF90AF900895D0
:10395000CF93DF93EC01DA016EBD0DB407FEFDCF0E
:103960008C918EBD1196EC91119782E090E00DB490
:1039700007FEFDCFEEBD22E08030920731F0FD0161
:10398000E80FF91FE0810196F2CF0DB407FEFDCFDD
:103990008FEF8EBD0DB407FEFDCF8FEF8EBD0DB442
:1039A00007FEFDCF8FEF8EBD0DB407FEFDCF8EB5A8
:1039B0008B838F71853011F481E006C083E18983A8
:1039C000CE010E942F1C80E0DF91CF9108950F93CC
:1039D0001F93CF93DF93EC018B010E94BF1BCE019D
:1039E00068E572E00E949C1B882361F0CE016CEFB9
:1039F000A8010E94A81C882329F0CE010E942F1C38
:103A000081E006C085E18983CE010E942F1C80E001
:103A1000DF91CF911F910F910895CF92DF92EF9296
:103A2000FF920F931F93CF93DF93EC017A018B01E9
:103A300069018C81833039F059E0EE0CFF1C001FC6
:103A4000111F5A95D1F7CE0168E1A80197010E9494
:103A5000DC1B882311F086E023C0CE016EEFA601A7
:103A60000E94A81C8823E9F0CE0168E572E00E945C
:103A70009C1B882311F487E113C0CE016DE020E088
:103A800030E040E050E00E94DC1B882341F48FEFDF
:103A90008EBD0DB407FEFDCF8EB5882379F086E18B
:103AA0008983CE010E942F1C80E0DF91CF911F916E
:103AB0000F91FF90EF90DF90CF900895CE010E947C
:103AC0002F1C81E0F2CFBF92CF92DF92EF92FF9254
:103AD0000F931F93CF93DF93EC016B017A010E9448
:103AE000753A8B01BB24BA9409C00E94753A601BD9
:103AF000710B6D52714010F081E10BC0BEBC0DB472
:103B000007FEFDCF8EB58B838F3F79F38E3F39F063
:103B10008FE08983CE010E942F1C80E030C0D70146
:103B20001197EF28D9F08FEF8EBD20E030E09FEFA6
:103B30000BC00DB407FEFDCF8EB59EBDF601E20FA2
:103B4000F31F80832F5F3F4F2A173B0790F30DB47D
:103B500007FEFDCF8EB5AC0DBD1D8C931B828FEF84
:103B60008EBD0DB407FEFDCF8EB58FEF8EBD0DB4AB
:103B700007FEFDCF8EB5CE010E942F1C81E0DF91A4
:103B8000CF911F910F91FF90EF90DF90CF90BF905A
:103B900008950F931F93CF93DF93EC018A0120E0E8
:103BA00030E040E050E00E94DC1B882339F080E1E7
:103BB0008983CE010E942F1C80E006C0CE01B8018F
:103BC00040E150E00E94631DDF91CF911F910F9162
:103BD0000895CF92DF92EF92FF920F931F93CF93AE
:103BE000DF93EC017A018B0169018C81833039F01C
:103BF000B9E0EE0CFF1C001F111FBA95D1F7CE01E2
:103C000061E1A80197010E94DC1B882339F084E060
:103C10008983CE010E942F1C80E006C0CE01B60130
:103C200040E052E00E94631DDF91CF911F910F9100
:103C3000FF90EF90DF90CF9008956F927F928F92D8
:103C40009F92AF92BF92CF92DF92EF92FF920F932B
:103C50001F93DF93CF93CDB7DEB760970FB6F8947D
:103C6000DEBF0FBECDBF5C016A017B013801490197
:103C700069E0AE014F5F5F4F0E94C91D882309F4C0
:103C800058C03B8536FD1EC0D401C3010196A11D5D
:103C9000B11D8C299D29AE29BF293F73330F2C8577
:103CA000221F2227221F322B232F30E040E050E03A
:103CB00082239323A423B5230097A105B10511F016
:103CC0008DE02FC0F5018481833071F009E0CC0CC8
:103CD000DD1CEE1CFF1C0A95D1F719E0660C771C61
:103CE000881C991C1A95D1F7C50160E2A7019601BD
:103CF0000E94DC1B882391F4C50161E2A4019301B9
:103D00000E94DC1B882351F4C50166E220E030E00C
:103D100040E050E00E94DC1B882321F18CE001C0D0
:103D20008EE0F501818305C0C5010E942F1C81E052
:103D300004C0C5010E942F1C80E060960FB6F89465
:103D4000DEBF0FBECDBFCF91DF911F910F91FF90CE
:103D5000EF90DF90CF90BF90AF909F908F907F902B
:103D60006F900895C50160E177E20E949C1B882353
:103D7000B9F2DACFBF92CF92DF92EF92FF920F9318
:103D80001F93CF93DF93EC01B62E1C8219824883D8
:103D90000E94753A6B01888161E00E94EA3A88814D
:103DA00061E00E94293B8AE061E00E94293B8AE0B1
:103DB00061E00E94EA3A8CE060E00E94EA3A8BE01F
:103DC00061E00E94EA3A8DE061E00E94EA3A8BE00D
:103DD0008A8382E58CBD1DBC80E09FEF9EBD0DB443
:103DE00007FEFDCF8F5F8A30C9F709C00E94753A80
:103DF0006C197D09615D774010F081E063C0CE01F0
:103E000060E020E030E040E050E00E94DC1B8130C8
:103E100069F71FEFCE0168E02AEA31E040E050E0A8
:103E20000E94DC1B853011F481E00DC080E01EBDD6
:103E30000DB407FEFDCF9EB58F5F8430C1F79B8325
:103E40009A3A31F482E08C838C81823051F40DC037
:103E50000E94753A6C197D09615D7740D8F282E065
:103E600031C0EE24FF2487010FC0E12CF12C012D7D
:103E700080E4182F09C00E94753A6C197D09615DB4
